:10000000830100308A0004288301F82A83129600B5
:10001000971B112817088A001608960A0319970AD1
:1000200082008313171883171608960A84000008A5
:10003000080043346C3465346134723420345334F2
:1000400063347234653465346E342E34003448348D
:1000500065346C346C346F3420344134673461342B
:1000600069346E3421340034483465346C346C3473
:100070006F34203457346F3472346C346434213428
:0200800000344A
:10047C00831292008610803E8312A12A831286106A
:10048C0001308312A1220230572A83128C000430CF
:10049C008D00FA30831257228D0B4F2A8C0B4D2A6C
:1004AC000800831292000430930053309400940B94
:1004BC005D2A930B5B2A920B592A0800831286142F
:1004CC00702A0D0897000C088C0A03198D0A062057
:1004DC008312A1220D0897000C080620003803197E
:1004EC000800672A831244228614842A1108970074
:1004FC001008900A0319910A0620A12211089700EE
:10050C00100806200038031908007C2A403083129A
:10051C003E228614992A110897001008900A031994
:10052C00910A0620A1221108970010080620003815
:10053C0003190800912A83129300F03995000608DC
:10054C000F391504860006140610130EF0399500A9
:10055C0006080F3915048600061406100D30940099
:10056C00940BB62A0800831290008614F03995007B
:10057C0006080F391504860006140610100EF03903
:10058C00950006080F3915048600061406100D3068
:10059C009100910BCF2A0800831286100F30831222
:1005AC0057223030860006140610053057220614E8
:1005BC00061021309000900BE12A0614061005302D
:1005CC008312572220308600061406100D3090003E
:1005DC00900BEE2A28308312A1220C30A122063077
:1005EC00A122792B83128E018E0A8F018C018C0A29
:1005FC008D0102308316850086018312D22234309D
:10060C0090000030910078228518102B06158C0173
:10061C008D010A2B06110D080C04031D0A2B8C01ED
:10062C008C0A8D018E0A03198F0A0E08023A0F04E8
:10063C00031D272B273090000030910083128C2251
:10064C000A2B0E08033A0F04031D2F2B831235239C
:10065C000A2B19309000003091008312092B831261
:10066C0044220030B9220330B9220530B9220530BA
:10067C00B9220530B9220030B9220330B92200303A
:10068C00B9220330B9220530B9220530B922003025
:10069C00B9220330B9220530B9220530B922033012
:1006AC00B92240303E222030B9220630B922053022
:1006BC00B9220030B9220330B9220530B9220230F8
:1006CC00B9222030B9220630B9220030B9220430C8
:1006DC00B9220130B9220730B9220430B9220130D5
:1006EC00B9220730B92A8312861040308312A12216
:1006FC0086140030A1220030A1220030A122043047
:10070C00A1220230A1221F30A1220230A1220430EA
:10071C00A1220030A1220030A1220030A1220430FD
:10072C00A1220830A1221F30A1220830A1220430BE
:10073C00A1220430A1220E30A1221530A1220430B6
:10074C00A1220C30A1221830A1220030A1220030AD
:10075C00A1220030A1220030A1220030A1220E30B3
:10076C00A1221130A1221130A1221130A1220E3070
:10077C00A1220030A1220030A1220030A1220E3093
:10078C00A1221130A1221530A1221130A1220E304C
:10079C00A1220030A1220030A1220030A122003081
:1007AC00A1220030A1221F30A1220030A122003052
:1007BC00A1220430A1220430A1220430A122043051
:1007CC00A1220630A1220330A1220030A122003048
:1007DC00A1220430A1220430A1220430A122043031
:1007EC00A1220C30A1221830A1220030A12200300D
:0407FC00A122442AC8
:02400E00F93F78
:00000001FF
